:020000040000FA
:020000000728CF
:04000A00003400348A
:02000E000730B9
:100010009F008316D73081008B0180308600FF302F
:100020008500831286011428851A1B28051A2A28A0
:1000300000308600142885182C2839203630860098
:1000400039203A3086003920393086003920353061
:100050008600142885181D2839203530860039205F
:100060003930860039203A30860039203630860013
:10007000142864300519C83085191430A10089305E
:0C008000A000A00B4128A10B3F280800A5
:02400E00503F21
:00000001FF
